:100000000C945E010C94D91F0C94AE1F0C94831FAA
:100010000C94581F0C942D1F0C94021F0C94D71E87
:100020000C94AC1E0C9491010C9491010C949101D0
:100030000C9491010C9491010C9491010C949101F8
:100040000C9491010C9491010C9491010C949101E8
:100050000C9491010C9491010C9491010C94621EEA
:100060000C9491010C942C1E0C94021E0C94910182
:100070000C9491010C9491010C9491010C94042026
:100080000C9491010C9491010C9491010C949101A8
:100090000C9491010C9491010C9491010C94910198
:1000A0000C9491010C9491010C9491010C94910188
:1000B0000C9491010C9491010C9491010C94910178
:1000C0000C9491010C9491010C9491010C94910168
:1000D0000C9491010C9491010C9491010C94910158
:1000E0000C9491010C9448030C94E2030C94360395
:1000F0000C944E030C945B040C94F81A0C94290293
:100100000C94C9030C9433040C9452030C94130301
:100110000C9444030C94BF200C94F1010C94061C25
:100120000C94BD1B0C9451040C94D11A0C94320302
:100130000C941A040C94F4030C941C1C0C94CB1B0C
:100140000C94C0010C94CF010C94C1030C94E301F6
:100150000C94B7040C947B020C9417030C94FC02CF
:100160000C943D040C94371B0C94911A0C9440038E
:100170000C94D8030C941B030C94FC030C940604FD
:100180000C9410040C943A030C9428030C9422034E
:100190000C9401030C9493010C94CE030C942C0347
:1001A0000C94EC030C941F030C94D21A0C94470487
:1001B0000C94290400002100240027002A002D00AF
:1001C0003000330001010000040107010A010000B2
:1001D0002200250028002B002E00310034000201EF
:1001E0000000050108010B010505050507050808C4
:1001F0000808020202020A0A0808040404040101B1
:1002000001010101010103030303030303030407C5
:1002100007070C0C0C0C0C0C0C0C0202020206065C
:100220000606060606060B0B0B0B0B0B0B0B01024F
:1002300010202008081020401020408002010201F8
:1002400008040201010204081020408080402010B0
:100250000804020180040201804020100804020109
:100260000804020101020408102040800102040871
:100270001020408000000A0B02090C0D0E08070335
:100280000401000000000000000000000000000069
:10029000000000000000000000000000000000005E
:1002A000121110000000000000000000000000001B
:1002B00000000000000000000000BF202092111F7D
:1002C00011241FBECFEFD1E2DEBFCDBF00E00CBFD7
:1002D00012E0A0E0B2E0E2E4FDE500E00BBF02C006
:1002E00007900D92A83AB107D9F72FE1A8EAB2E03A
:1002F00001C01D92A131B207E1F711E0CEE5D1E0D6
:1003000000E006C021970109802FFE010E94A22C67
:10031000CD35D10780E00807A9F70E9414210C947D
:100320009F2E0C940000AF92BF92CF92DF92EF927B
:10033000FF920F931F93CF93DF936C017B018B018F
:10034000040F151FEB015E01AE18BF08C017D107DF
:1003500059F06991D601ED91FC910190F081E02D69
:10036000C6011995892B79F7C501DF91CF911F91AE
:100370000F91FF90EF90DF90CF90BF90AF900895D6
:10038000FC01538D448D252F30E0842F90E0821B9B
:10039000930B541710F0CF96089501970895FC0120
:1003A000918D828D981761F0A28DAE0FBF2FB11D78
:1003B0005D968C91928D9F5F9F73928F90E00895D0
:1003C0008FEF9FEF0895FC01918D828D981731F08A
:1003D000828DE80FF11D858D90E008958FEF9FEFDE
:1003E0000895FC01918D228D892F90E0805C9F4FB4
:1003F000821B91098F739927089581E59EE10E94E0
:10040000F10121E0892B09F420E0822F0895FC01FD
:10041000A48DA80FB92FB11DA35ABF4F2C91848D65
:1004200090E001968F739927848FA689B7892C93C2
:10043000A089B1898C91837080648C93938D848D15
:10044000981306C00288F389E02D80818F7D808318
:100450000895EF92FF920F931F93CF93DF93EC01D8
:1004600081E0888F9B8D8C8D98131AC0E889F9895B
:10047000808185FF15C09FB7F894EE89FF8960835E
:10048000E889F98980818370806480839FBF81E0DF
:1004900090E0DF91CF911F910F91FF90EF90089521
:1004A000F62E0B8D10E00F5F1F4F0F731127E02EFC
:1004B0008C8D8E110CC00FB607FCFACFE889F98934
:1004C000808185FFF5CFCE010E940702F1CFEB8D31
:1004D000EC0FFD2FF11DE35AFF4FF0829FB7F89408
:1004E0000B8FEA89FB8980818062CFCF682F81E5FD
:1004F0009EE10C942902CF93DF93EC01888D882331
:10050000B9F0AA89BB89E889F9898C9185FD03C076
:10051000808186FD0DC00FB607FCF7CF8C9185FF5B
:10052000F2CF808185FFEDCFCE010E940702E9CF97
:10053000DF91CF91089580E090E0892B29F00E940F
:10054000FD0181110E94000080E090E0892B49F0BC
:1005500080E090E0892B29F00E94000081110E9428
:10056000000080E090E0892B49F080E090E0892B4A
:1005700029F00E94000081110E94000080E090E0BC
:10058000892B49F080E090E0892B29F00E9400003F
:1005900081110C9400000895282F30E0F901EC58E7
:1005A000FD4F9491F901E25DFD4F449128513E4F7A
:1005B000F9012491222309F435C0992311F19150B6
:1005C0009231F8F4E92FF0E08827E651FD4F8F4F84
:1005D0000C94A22C1B031F03FC021303170301033B
:1005E000220328032C03320336033A034003440357
:1005F000010348034E035203809180008F7780935C
:100600008000E22FF0E0EE0FFF1FE253FE4FA591B6
:10061000B4918FB7F894EC91611148C040954E2386
:100620004C938FBF0895809180008F7DE8CF80919B
:100630008000877FE4CF84B58F7784BDE2CF84B517
:100640008F7DFBCF8091B0008F778093B000D9CFA2
:100650008091B0008F7DF9CF809190008F7780934B
:100660009000CFCF809190008F7DF9CF8091900046
:10067000877FF5CF8091A0008F778093A000C1CFB6
:100680008091A0008F7DF9CF8091A000877FF5CF6A
:10069000809120018F7780932001B3CF809120013A
:1006A0008F7DF9CF80912001877FF5CF4E2BB8CF7A
:1006B000CF93DF9390E0FC01E25DFD4F24918851E0
:1006C0009E4FFC0184918823D1F090E0880F991F00
:1006D000FC01EC54FE4FA591B491FC01E253FE4F96
:1006E000C591D49161110EC09FB7F8948C91E22FFF
:1006F000E0958E238C932881E223E8839FBFDF91CE
:10070000CF9108958FB7F894EC91E22BEC938FBFC3
:10071000F6CF1F93CF93DF93182FEB0161E00E9478
:100720005803209739F460E0812FDF91CF911F911A
:100730000C94CC02CF3FD10511F461E0F5CFE12F4D
:10074000F0E0EC58FD4FE491E150E23108F0B3C025
:10075000F0E08827E155FC4F8F4F0C94A22CC10389
:10076000C903CE03D803E2035B04EC03F403FC03E8
:10077000060410041A04290433045B043D044704EE
:10078000510484B5806884BDC7BDDF91CF911F91AE
:10079000089584B5806284BDC8BDF7CF8091800084
:1007A000806880938000D0938900C0938800EDCF4B
:1007B00080918000806280938000D0938B00C093F2
:1007C0008A00E3CF80918000886080938000D0937E
:1007D0008D00C0938C00D9CF8091B0008068809349
:1007E000B000C093B300D1CF8091B00080628093FD
:1007F000B000C093B400C9CF80919000806880930E
:100800009000D0939900C0939800BFCF8091900042
:10081000806280939000D0939B00C0939A00B5CFE4
:1008200080919000886080939000D0939D00C09349
:100830009C00ABCF8091A00080688093A000809145
:10084000A0008F7B8093A000D093A900C093A80044
:100850009CCF8091A00080628093A000D093AB00D9
:10086000C093AA0092CF8091A00088608093A000DE
:10087000D093AD00C093AC0088CF809120018068F8
:1008800080932001D0932901C09328017ECF8091CD
:100890002001806280932001D0932B01C0932A0114
:1008A00074CF80912001886080932001D0932D0126
:1008B000C0932C016ACFC038D1050CF03ECF33CFA6
:1008C0003FB7F8948091B4029091B502A091B6021E
:1008D000B091B70226B5A89B05C02F3F19F001962D
:1008E000A11DB11D3FBFBA2FA92F982F8827BC018A
:1008F000CD01620F711D811D911D42E0660F771FB2
:10090000881F991F4A95D1F708958F929F92AF92B1
:10091000BF92CF92DF92EF92FF924B015C010E9457
:1009200060046B017C010E9460046C197D098E09D2
:100930009F09683E734081059105A8F321E0821A62
:100940009108A108B10888EEC80E83E0D81EE11C0A
:10095000F11C81149104A104B10429F7FF90EF90D8
:10096000DF90CF90BF90AF909F908F9008950895A3
:100970008091200A9091210AA091220AB091230A25
:10098000892B8A2B8B2BE1F080911C0A90911D0AF8
:10099000A0911E0AB0911F0A892B8A2B8B2B81F004
:1009A00080911602909117028F3F910549F0809136
:1009B0001A0A90911B0A892B19F0109213020895BC
:1009C00081E0809313020895CF93DF9380EC90E051
:1009D0000E94760290E080E00E947602CEE1D3E0B1
:1009E0002091AA023091AB02CE018E519340821722
:1009F0009307A8F46991603C51F48BED90E00E945C
:100A000076026CED81E59EE10E942902E9CF6B3D03
:100A1000C9F78BED90E00E9476026DEDF3CF80EC8C
:100A200090E00E9476021092AB021092AA02DF912F
:100A3000CF91089580EC90E00E94760283E090E0F0
:100A40000E9476026091160281E59EE10E942902D1
:100A500080EC90E00C94760280EC90E00E947602AC
:100A600085E090E00E9476026091140281E59EE1AB
:100A70000E94290280EC90E00C94760280EC90E0D9
:100A80000E94760284E090E00E94760260911A0A49
:100A900081E59EE10E94290280EC90E00C947602B0
:100AA000CF93C82F80EC90E00E94760280E990E01E
:100AB0000E9476026C2F81E59EE10E94290280EC63
:100AC00090E0CF910C947602803C51F48BED90E055
:100AD0000E9476028CED682F81E59EE10C9429023C
:100AE0008B3DC9F78BED90E00E9476028DEDF3CF40
:100AF0001F93CF93DF9380EC90E00E94760281E019
:100B000090E00E947602C091200AD091210A1091B3
:100B1000220A8091230A0E946405812F0E946405A5
:100B20008D2F0E9464058C2F0E94640580EC90E05C
:100B3000DF91CF911F910C9476021F93CF93DF9397
:100B400080EC90E00E94760282E090E00E947602C3
:100B5000C0911C0AD0911D0A10911E0A80911F0A93
:100B60000E946405812F0E9464058D2F0E946405F8
:100B70008C2F0E94640580EC90E0DF91CF911F9153
:100B80000C94760280EC90E00E94760284E290E081
:100B90000E9476028091A9020E94640580EC90E098
:100BA0000C947602CF93C0910102C35680EC90E082
:100BB0000E94760283E290E00E9476028C2F0E94CF
:100BC000640580EC90E0CF910C94760260E08DE0BB
:100BD0000C94CC0261E08DE00C94CC02CF93DF93B7
:100BE000EC0161E08DE00E94CC020E94E60564E623
:100BF00070E080E090E00E9485040E94EA0564E6CF
:100C000070E080E090E00E948504219771F7DF9109
:100C1000CF910C94E60560E08CE00C94CC020F932D
:100C20001F93CF93DF938C01EC01892B11F4C1E06A
:100C3000D0E00E940B0664E670E080E090E00E9445
:100C4000850461E08CE00E94CC0264E670E080E004
:100C500090E00E9485040115110559F3219749F789
:100C6000DF91CF911F910F910C940B060E94EA0522
:100C70000E940B066AE070E080E090E00E9485042C
:100C800061E08CE00E94CC020E94E60565E070E025
:100C900080E090E00E948504E9CF0F931F93CF93EB
:100CA000DF938C01EC01892B11F4C1E0D0E061E00D
:100CB0008CE00E94CC0260E08DE00E94CC0264E6F1
:100CC00070E080E090E00E94850460E08CE00E948B
:100CD000CC0261E08DE00E94CC0264E670E080E02E
:100CE00090E00E9485040115110509F32197F9F69A
:100CF0000E940B06DF91CF911F910F910C94E60596
:100D00002F923F924F925F926F927F928F929F921B
:100D1000AF92BF92CF92DF92EF92FF920F931F9309
:100D2000CF93DF93CDB7DEB7C857D1090FB6F8948C
:100D3000DEBF0FBECDBFE9969FAF8EAFE9971A0118
:100D4000DC0118960D911D912D913C911B97619698
:100D50000CAF1DAF2EAF3FAF61971C960D911D914B
:100D60002D913C911F9709831A832B833C835096C6
:100D70000D911D912D913C9153970D831E832F83CF
:100D8000388754960D911D912D913C915797098765
:100D90001A872B873C87E6966FAFE697E7967FAF7B
:100DA000E797A85ABF4F6396BFAFAEAF6397FC01FA
:100DB000E45AFF4F6596FFAFEEAF65978C01005A7E
:100DC0001F4F67961FAF0EAF67979C012C593F4F7F
:100DD00069963FAF2EAF699788599F4F6B969FAF2B
:100DE0008EAF6B97E996AEADBFADE997A459BF4FF3
:100DF0006D96BFAFAEAF6D97E996EEADFFADE997DB
:100E0000E059FF4F6F96FFAFEEAF6F97E9960EADCB
:100E10001FADE9970C581F4FA1961FAF0EAFA197BA
:100E2000E9962EAD3FADE99728583F4FA3963FAFC7
:100E30002EAFA397E9968EAD9FADE99784589F4F4B
:100E4000A5969FAF8EAFA597E996AEADBFADE997DA
:100E5000A058BF4FA796BFAFAEAFA797E996EEAD2C
:100E6000FFADE997EC57FF4FA996FFAFEEAFA997FB
:100E7000E9960EAD1FADE99708571F4FAB961FAF10
:100E80000EAFAB97E9962EAD3FADE99724573F4F94
:100E9000AD963FAF2EAFAD97E9968EAD9FADE9977A
:100EA00080579F4FAF969FAF8EAFAF97E996AEAD8D
:100EB000BFADE997AC56BF4FE196BFAFAEAFE1977C
:100EC000E796AEADBFADE7970D911D912D913C9189
:100ED0000D871E872F87388B6396EEADFFAD639726
:100EE000008311832283338361968CAD9DADAEADBB
:100EF000BFAD619788589B45A549B842800F911FA7
:100F0000A21FB31F4D815E816F81788509851A8587
:100F10002B853C85402751276227732709811A8139
:100F20002B813C81402351236223732309851A8539
:100F30002B853C854027512762277327840F951FF7
:100F4000A61FB71F8C019D0147E0000F111F221F34
:100F5000331F4A95D1F7AC01BD01E9E1769567955C
:100F600057954795EA95D1F7402B512B622B732B60
:100F700089819A81AB81BC81480F591F6A1F7B1FF1
:100F8000E796AEADBFADE79714960D911D912D91EB
:100F90003C911797098B1A8B2B8B3C8B6596EEAD8A
:100FA000FFAD6597008311832283338389859A85FA
:100FB000AB85BC858A5A9844A843B741800F911FDE
:100FC000A21FB31FC980DA80EB80FC800D811E81D7
:100FD0002F813885C026D126E226F326C422D522C9
:100FE000E622F722C026D126E226F3268C0D9D1D8F
:100FF000AE1DBF1D8C019D01FCE0000F111F221FC3
:10100000331FFA95D1F76C017D01A4E1F694E794C2
:10101000D794C794AA95D1F7C02AD12AE22AF32AF5
:10102000C40ED51EE61EF71EE796AEADBFADE79720
:1010300018968D919D910D90BC91A02D8D8B9E8BBE
:10104000AF8BB88F6796EEADFFAD679780839183C6
:10105000A283B3838D819E81AF81B88585529F48DD
:10106000AF4DBB4D0D891E892F89388D800F911F83
:10107000A21FB31F49805A806B807C80442655266E
:10108000662677264C205D206E207F2009811A81FC
:101090002B813C814026512662267326840D951DA6
:1010A000A61DB71D8C019D01EFE03695279517957C
:1010B0000795EA95D1F72C013D01F1E1440C551C4F
:1010C000661C771CFA95D1F7402A512A622A732AA6
:1010D0004C0C5D1C6E1C7F1CE796AEADBFADE79758
:1010E0001C968D919D910D90BC91A02D898F9A8F0A
:1010F000AB8FBC8F6996EEADFFAD6997808391830E
:10110000A283B38389819A81AB81BC81825191434F
:10111000A244BE43098D1A8D2B8D3C8D800F911FEB
:10112000A21FB31F8A019B010C251D252E253F25DB
:1011300004211521262137210427152726273727A3
:10114000800F911FA21FB31F4C015D011AE0B694DE
:10115000A794979487941A95D1F78C019D0186E105
:10116000000F111F221F331F8A95D1F70829192953
:101170002A293B29040D151D261D371DE796AEAD06
:10118000BFADE79750968D919D910D90BC91A02D8C
:101190008D8F9E8FAF8FB8A36B96EEADFFAD6B9723
:1011A00080839183A283B3838155904FA348BA4033
:1011B000840F951FA61FB71FB701A601442555250B
:1011C0006625772540235123622373234C255D2513
:1011D0006E257F25840F951FA61FB71F4C015D014B
:1011E00047E0880C991CAA1CBB1C4A95D1F7AC019E
:1011F000BD01E9E17695679557954795EA95D1F751
:10120000482959296A297B29400F511F621F731FE2
:10121000E796AEADBFADE79754968D919D910D9039
:10122000BC91A02D89A39AA3ABA3BCA36D96EEADF0
:10123000FFAD6D9780839183A283B383865D9943CD
:10124000A847B84B8C0D9D1DAE1DBF1D73016201DB
:10125000C026D126E226F326C422D522E622F72292
:10126000C424D524E624F7248C0D9D1DAE1DBF1D7E
:101270004C015D01FCE0880C991CAA1CBB1CFA9572
:10128000D1F76C017D01A4E1F694E794D794C7945B
:10129000AA95D1F7C828D928EA28FB28C40ED51E5C
:1012A000E61EF71EE796AEADBFADE79758968D9157
:1012B0009D910D90BC91A02D8DA39EA3AFA3B8A727
:1012C0006F96EEADFFAD6F9780839183A283B3835A
:1012D0008D5E994BAF4CB745840D951DA61DB71D6E
:1012E0002801390144265526662677264C205D20A4
:1012F0006E207F204026512662267326840D951D80
:10130000A61DB71D4C015D01EFE0B694A79497941C
:101310008794EA95D1F72C013D01F1E1440C551C6D
:10132000661C771CFA95D1F7482859286A287B282B
:101330004C0C5D1C6E1C7F1CE796AEADBFADE797F5
:101340005C968D919D910D90BC91A02D89A79AA737
:10135000ABA7BCA7A196EEADFFADA197808391830B
:10136000A283B3838F5F9A46A94BB240800F911F2F
:10137000A21FB31F8A019B010C251D252E253F2589
:101380000421152126213721042715272627372751
:10139000800F911FA21FB31F4C015D011AE0B6948C
:1013A000A794979487941A95D1F78C019D0186E1B3
:1013B000000F111F221F331F8A95D1F70829192901
:1013C0002A293B29040D151D261D371DE796AEADB4
:1013D000BFADE79790968D919D910D90BC91A02DFA
:1013E0008DA79EA7AFA7B8ABA396EEADFFADA39711
:1013F00080839183A283B38388529746AF47B649CF
:10140000840F951FA61FB71FB701A60144255525B8
:101410006625772540235123622373234C255D25C0
:101420006E257F25840F951FA61FB71F4C015D01F8
:1014300047E0880C991CAA1CBB1C4A95D1F7AC014B
:10144000BD01E9E17695679557954795EA95D1F7FE
:10145000482959296A297B29400F511F621F731F90
:10146000E796AEADBFADE79794968D919D910D90A7
:10147000BC91A02D89AB9AABABABBCABA596EEAD46
:10148000FFADA59780839183A283B3838155984054
:10149000AB4BB4478C0D9D1DAE1DBF1D730162018A
:1014A000C026D126E226F326C422D522E622F72240
:1014B000C424D524E624F7248C0D9D1DAE1DBF1D2C
:1014C0004C015D01FCE0880C991CAA1CBB1CFA9520
:1014D000D1F76C017D01A4E1F694E794D794C79409
:1014E000AA95D1F7C828D928EA28FB28C40ED51E0A
:1014F000E61EF71EE796AEADBFADE79798968D91C5
:101500009D910D90BC91A02D8DAB9EABAFABB8AFB4
:10151000A796EEADFFADA79780839183A283B38397
:101520008F54944AA109B109840D951DA61DB71DBC
:101530002801390144265526662677264C205D2051
:101540006E207F204026512662267326840D951D2D
:10155000A61DB71D4C015D01EFE0B694A7949794CA
:101560008794EA95D1F72C013D01F1E1440C551C1B
:10157000661C771CFA95D1F7482859286A287B28D9
:101580004C0C5D1C6E1C7F1CE796AEADBFADE797A3
:101590009C968D919D910D90BC91A02D89AF9AAF95
:1015A000ABAFBCAFA996EEADFFADA9978083918399
:1015B000A283B38382549842A34AB647800F911FF7
:1015C000A21FB31F8A019B010C251D252E253F2537
:1015D00004211521262137210427152726273727FF
:1015E000800F911FA21FB31F4C015D011AE0B6943A
:1015F000A794979487941A95D1F78C019D0186E161
:10160000000F111F221F331F8A95D1F708291929AE
:101610002A293B29040D151D261D371DE796AEAD61
:10162000BFADE797D0968D919D910D90BC91A02D67
:1016300021968CAF9DAFAEAFBFAF2197AB96EEAD0D
:10164000FFADAB9780839183A283B3834C015D018F
:10165000FEED8F1AFEEE9F0AFFE6AF0AF4E9BF0A1D
:10166000840E951EA61EB71EB701A601442555255A
:101670006625772540235123622373234C255D255E
:101680006E257F25480D591D6A1D7B1D4A015B0192
:1016900097E0880C991CAA1CBB1C9A95D1F7E9E12C
:1016A0007695679557954795EA95D1F74829592931
:1016B0006A297B29400F511F621F731FE796AEAD49
:1016C000BFADE797D4968D919D910D90BC91A02DC3
:1016D00025968CAF9DAFAEAFBFAF2597AD96EEAD63
:1016E000FFADAD9780839183A283B3834C015D01ED
:1016F000FDE68F1AFEE89F0AF7E6AF0AF2E0BF0A9E
:101700008C0C9D1CAE1CBF1C73016201C026D1262F
:10171000E226F326C422D522E622F722C424D524C9
:10172000E624F724C80CD91CEA1CFB1C460157010F
:10173000FCE0880C991CAA1CBB1CFA95D1F7A4E10B
:10174000F694E794D794C794AA95D1F7C828D928D6
:10175000EA28FB28C40ED51EE61EF71EE796AEAD9E
:10176000BFADE797D8968D919D910D90BC91A02D1E
:1017700029968CAF9DAFAEAFBFAF2997AF96EEADB8
:10178000FFADAF9780839183A283B3834C015D014A
:10179000F2E78F1AFCEB9F0AF6E8AF0AF9E5BF0AF9
:1017A000840C951CA61CB71C28013901442655261B
:1017B000662677264C205D206E207F20402651260D
:1017C00062267326480C591C6A1C7B1C530142017B
:1017D000BFE0B694A79497948794BA95D1F781E126
:1017E000440C551C661C771C8A95D1F7482859284B
:1017F0006A287B284C0C5D1C6E1C7F1CE796AEADE6
:10180000BFADE797DC968D919D910D90BC91A02D79
:101810002D968CAF9DAFAEAFBFAF2D97E196EEADDD
:10182000FFADE19780839183A283B3834C015D0177
:10183000FFED8F1AF7EF9F0AFBE4AF0AF6EBBF0A42
:10184000800E911EA21EB31E8A019B010C251D2530
:101850002E253F2504211521262137210427152770
:1018600026273727080D191D2A1D3B1D4801590140
:101870009AE0B694A794979487949A95D1F7E6E165
:10188000000F111F221F331FEA95D1F708291929CC
:101890002A293B29040D151D261D371D89889A8884
:1018A000AB88BC888EE9881A8AED980A81EEA80A6E
:1018B00089E0B80A840E951EA61EB71EB301A201C8
:1018C00040275127622773274C215D216E217F21FC
:1018D0004425552566257725480D591D6A1D7B1D14
:1018E0004A015B01F5E0880C991CAA1CBB1CFA9507
:1018F000D1F7ABE17695679557954795AA95D1F7BE
:10190000482959296A297B29400F511F621F731FDB
:101910008DA09EA0AFA0B8A490EC891A9CE4990A6F
:101920009FEBA90A9FE3B90A8C0C9D1CAE1CBF1C3F
:1019300068017901C426D526E626F726C420D520DD
:10194000E620F720C026D126E226F326C80CD91CB3
:10195000EA1CFB1C46015701B9E0880C991CAA1C23
:10196000BB1CBA95D1F787E1F694E794D794C79456
:101970008A95D1F7C828D928EA28FB28C40ED51E95
:10198000E61EF71E89AC9AACABACBCACAFEA8A1AC7
:10199000A5EA9A0AA1EAAA0AA9EDBA0A840C951C3A
:1019A000A61CB71C2A013B014C245D246E247F2415
:1019B000402251226222732244265526662677262B
:1019C000480C591C6A1C7B1C530142019EE0880C88
:1019D000991CAA1CBB1C9A95D1F7E2E176946794F6
:1019E00057944794EA95D1F7482859286A287B28C4
:1019F0004C0C5D1C6E1C7F1C8D849E84AF84B8884B
:101A0000B6E58B1AB8E39B0AB9E4AB0AB6E1BB0AA8
:101A1000800E911EA21EB31E970186010425152576
:101A20002625372504231523262337230C251D259A
:101A30002E253F25080D191D2A1D3B1D4801590162
:101A4000FCE0B694A79497948794FA95D1F7A4E113
:101A5000000F111F221F331FAA95D1F7082919293A
:101A60002A293B29040D151D261D371D89A09AA082
:101A7000ABA0BCA0E3EA8E1AEFEE9E0AE0EDAE0A40
:101A8000E9E2BE0A840E951EA61EB71EB301A2018E
:101A900040275127622773274C215D216E217F212A
:101AA0004425552566257725480D591D6A1D7B1D42
:101AB0004A015B01B5E0880C991CAA1CBB1CBA95B5
:101AC000D1F78BE176956795579547958A95D1F72C
:101AD000482959296A297B29400F511F621F731F0A
:101AE0008DA89EA8AFA8B8ACFDEA8F1AFBEE9F0A9E
:101AF000FBEBAF0AFDEFBF0A8C0C9D1CAE1CBF1C9C
:101B000068017901C426D526E626F726C420D5200B
:101B1000E620F720C026D126E226F326C80CD91CE1
:101B2000EA1CFB1C4601570199E0880C991CAA1C71
:101B3000BB1C9A95D1F7E7E1F694E794D794C79444
:101B4000EA95D1F7C828D928EA28FB28C40ED51E63
:101B5000E61EF71E2D968CAC9DACAEACBFAC2D979F
:101B60008FE7881A89E1980A8EE5A80A87E2B80A01
:101B7000840C951CA61CB71C2A013B014C245D2437
:101B80006E247F244022512262227322442655264D
:101B900066267726480C591C6A1C7B1C530142019F
:101BA000FEE0880C991CAA1CBB1CFA95D1F7A2E197
:101BB0007694679457944794AA95D1F74828592862
:101BC0006A287B284C0C5D1C6E1C7F1C8D8C9E8CA7
:101BD000AF8CB8A098E3891A94E0990A9CE2A90A0C
:101BE00098E1B90A800E911EA21EB31E97018601CC
:101BF00004251525262537250423152326233723D9
:101C00000C251D252E253F25080D191D2A1D3B1DC0
:101C100048015901BCE0B694A79497948794BA956B
:101C2000D1F784E1000F111F221F331F8A95D1F7CE
:101C3000082919292A293B29040D151D261D371DA0
:101C400089A89AA8ABA8BCA8AAE18A1AA2E39A0A12
:101C5000AEE1AA0AAEEDBA0A840E951EA61EB71E04
:101C6000B301A20140275127622773274C215D2130
:101C70006E217F214425552566257725480D591D60
:101C80006A1D7B1D4A015B0195E0880C991CAA1C0A
:101C9000BB1C9A95D1F7EBE17695679557954795DB
:101CA000EA95D1F7482959296A297B29400F511F04
:101CB000621F731F29968CAC9DACAEACBFAC29974C
:101CC000BAE28B1AB8EF9B0AB8ECAB0ABCE3BB0ACA
:101CD0008C0C9D1CAE1CBF1C68017901C426D52646
:101CE000E626F726C420D520E620F720C026D126F8
:101CF000E226F326C80CD91CEA1CFB1C460157013E
:101D0000F9E0880C991CAA1CBB1CFA95D1F7A7E135
:101D1000F694E794D794C794AA95D1F7C828D92800
:101D2000EA28FB28C40ED51EE61EF71E898C9A8C65
:101D3000AB8CBC8CE9E78E1AE2EF9E0AEAE2AE0AAF
:101D4000EBE0BE0A840C951CA61CB71C2A013B01C3
:101D50004C245D246E247F2440225122622273226F
:101D60004426552666267726480C591C6A1C7B1C7F
:101D700053014201BEE0880C991CAA1CBB1CBA95F9
:101D8000D1F782E176946794579447948A95D1F776
:101D9000482859286A287B284C0C5D1C6E1C7F1C27
:101DA0008DA49EA4AFA4B8A8F3E18F1AFBEE9F0AFE
:101DB000F5EAAF0AFAEBBF0A800E911EA21EB31E0F
:101DC000970186010425152526253725042315238B
:101DD000262337230C251D252E253F25080D191DEB
:101DE0002A1D3B1D480159019CE0B694A794979485
:101DF00087949A95D1F7E4E1000F111F221F331F3A
:101E0000EA95D1F7082919292A293B29040D151D1E
:101E1000261D371D25968CAC9DACAEACBFAC25976E
:101E20008BEF881A86E1980A8CE1A80A86E5B80A41
:101E3000840E951EA61EB71EB301A201402751278E
:101E4000622773274C215D216E217F214425552572
:101E500066257725480D591D6A1D7B1D4A015B01CA
:101E6000F5E0880C991CAA1CBB1CFA95D1F7ABE1D4
:101E70007695679557954795AA95D1F74829592999
:101E80006A297B29400F511F621F731F8D889E880E
:101E9000AF88B88C98E0891A9CE5990A90E1A90A64
:101EA00093E0B90A8C0C9D1CAE1CBF1C6801790123
:101EB000C426D526E626F726C420D520E620F7201E
:101EC000C026D126E226F326C80CD91CEA1CFB1C2E
:101ED00046015701B9E0880C991CAA1CBB1CBA9595
:101EE000D1F787E1F694E794D794C7948A95D1F710
:101EF000C828D928EA28FB28C40ED51EE61EF71EDE
:101F000089A49AA4ABA4BCA4A7E28A1AADEF9A0A4A
:101F1000A0E9AA0AA8E9BA0A840C951CA61CB71C59
:101F20002A013B014C245D246E247F24402251224F
:101F3000622273224426552666267726480C591CB1
:101F40006A1C7B1C530142019EE0880C991CAA1C50
:101F5000BB1C9A95D1F7E2E1769467945794479425
:101F6000EA95D1F7482859286A287B284C0C5D1C33
:101F70006E1C7F1C4601570184249524A624B72497
:101F800021968CAD9DADAEADBFAD21978657934BDD
:101F9000A54DB247800F911FA21FB31F9501840169
:101FA00004231523262337230C251D252E253F2505
:101FB000800F911FA21FB31F8C019D01FCE036957D
:101FC000279517950795FA95D1F7E5960CAF1DAFB4
:101FD0002EAF3FAFE5978C019D01A4E1000F111FCB
:101FE000221F331FAA95D1F7E5968CAD9DADAEADFE
:101FF000BFADE597082B192B2A2B3B2B040D151D84
:10200000261D371D89A19AA1ABA1BCA18E5B964C60
:10201000A540B109840F951FA61FB71F80269126E2
:10202000A226B326880E991EAA1EBB1ED501C40186
:1020300044E0880F991FAA1FBB1F4A95D1F75CE1A6
:10204000B694A794979487945A95D1F7882A992A99
:10205000AA2ABB2A800E911EA21EB31E4DA55EA504
:102060006FA578A94F5759406E4878474C0D5D1DB4
:102070006E1D7F1D73016201C026D126E226F32664
:10208000C824D924EA24FB24C40ED51EE61EF71E5C
:10209000B701A601EBE0440F551F661F771FEA95B5
:1020A000D1F7F5E1F694E794D794C794FA95D1F770
:1020B000C42AD52AE62AF72AC80CD91CEA1CFB1C1C
:1020C00049AD5AAD6BAD7CAD4E5D5E49624672491D
:1020D000440E551E661E771EB901A80148255925D4
:1020E0006A257B254C255D256E257F25440E551ED2
:1020F000661E771ED20123013D014C0C5D1C6E1C37
:102100007F1C29964CAD5DAD6EAD7FAD2997445FC8
:10211000574C6A417240400F511F621F731F950157
:1021200084010C251D252E253F2504251525262552
:102130003725040F151F261F371FB901A801A9E075
:102140007695679557954795AA95D1F7B7E1000F12
:10215000111F221F331FBA95D1F7042B152B262BE5
:10216000372B040D151D261D371D49895A896B898A
:102170007C894C5B554161447B45480D591D6A1D66
:102180007B1D4601570184249524A624B72480266C
:102190009126A226B326840E951EA61EB71EB50153
:1021A000A40184E0440F551F661F771F8A95D1F75D
:1021B0009CE1B694A794979487949A95D1F7842A32
:1021C000952AA62AB72A800E911EA21EB31E4D8DF7
:1021D0005E8D6F8D78A1475550436142744BC40E9C
:1021E000D51EE61EF71EB301A20140275127622724
:1021F0007327482559256A257B254C0D5D1D6E1DCD
:102200007F1DDB01CA01EBE0880F991FAA1FBB1FCE
:10221000EA95D1F7F5E17695679557954795FA9543
:10222000D1F7482B592B6A2B7B2B480D591D6A1D62
:102230007B1DC9A4DAA4EBA4FCA4B0EACB1AB4EBCE
:10224000DB0AB4E4EB0AB9E0FB0A4C0C5D1C6E1C23
:102250007F1C68017901C824D924EA24FB24C42600
:10226000D526E626F7264C0C5D1C6E1C7F1CF20161
:1022700023013F01440E551E661E771ECDA8DEA821
:10228000EFA8F8ACF0E9CF1AF3E4DF0AF0E4EF0AC4
:10229000F1E4FF0AC00ED11EE21EF31E9501840177
:1022A0000427152726273727042515252625372512
:1022B0000C0D1D1D2E1D3F1D68017901A9E0F6942E
:1022C000E794D794C794AA95D1F7B7E1000F111FEF
:1022D000221F331FBA95D1F70C291D292E293F291A
:1022E000040D151D261D371D2596CCACDDACEEACBE
:1022F000FFAC25978AE3C81A81E8D80A84E6E80A81
:1023000087EDF80AC80CD91CEA1CFB1C4A015B01CA
:1023100084249524A624B72480269126A226B326B9
:102320008C0C9D1CAE1CBF1C7501640184E0CC0CA0
:10233000DD1CEE1CFF1C8A95D1F79CE1B694A79496
:10234000979487949A95D1F78C289D28AE28BF281A
:10235000800E911EA21EB31ECD84DE84EF84F88809
:1023600096E0C91A98EDD90A9EE5E90A95E1F90ABD
:10237000C40ED51EE61EF71EB301A2014027512749
:1023800062277327482559256A257B254C0D5D1D3D
:102390006E1D7F1D6A017B01EBE0CC0CDD1CEE1C89
:1023A000FF1CEA95D1F7F5E1769567955795479526
:1023B000FA95D1F74C295D296E297F29480D591DC1
:1023C0006A1D7B1DC98CDA8CEB8CFC8CABE7CA1ABE
:1023D000AFECDA0AA0E1EA0AABE2FA0A4C0C5D1CA7
:1023E0006E1C7F1C68017901C824D924EA24FB24CF
:1023F000C426D526E626F7264C0C5D1C6E1C7F1CD9
:10240000F20123013F01440E551E661E771ECDA02A
:10241000DEA0EFA0F8A4FBEFCF1AF2EEDF0AF7E799
:10242000EF0AFBEFFF0AC00ED11EE21EF31E95015C
:102430008401042715272627372704251525262557
:1024400037250C0D1D1D2E1D3F1D68017901A9E0CA
:10245000F694E794D794C794AA95D1F7B7E1000F03
:10246000111F221F331FBA95D1F70C291D292E29C0
:102470003F29040D151D261D371DC9A8DAA8EBA894
:10248000FCA887ECC81A8FE2D80A8BE2E80A86E239
:10249000F80AC80CD91CEA1CFB1C4A015B01842405
:1024A0009524A624B72480269126A226B3268C0C38
:1024B0009D1CAE1CBF1C7501640184E0CC0CDD1CAE
:1024C000EE1CFF1C8A95D1F79CE1B694A7949794D3
:1024D00087949A95D1F78C289D28AE28BF28800E26
:1024E000911EA21EB31E2196CCACDDACEEACFFACAF
:1024F00021979BE1C91A96E6D90A94E2E90A99E183
:10250000F90AC40ED51EE61EF71EB301A20140272C
:10251000512762277327482559256A257B254C0DAD
:102520005D1D6E1D7F1D6A017B01EBE0CC0CDD1C87
:10253000EE1CFF1CEA95D1F7F5E176956795579566
:102540004795FA95D1F74C295D296E297F29480DC9
:10255000591D6A1D7B1D2D96CCACDDACEEACFFACDD
:102560002D97A8E0CA1AA3E8DA0AADE5EA0AA0EEB8
:10257000FA0A4C0C5D1C6E1C7F1C68017901C82492
:10258000D924EA24FB24C426D526E626F7264C0CBB
:102590005D1C6E1C7F1CF20123013F01440E551E81
:1025A000661E771ECD88DE88EF88F88CFBE9CF1A8F
:1025B000F9EADF0AF3E5EF0AFBE3FF0AC00ED11EDA
:1025C000E21EF31E950184010427152726273727CD
:1025D00004251525262537250C0D1D1D2E1D3F1DF7
:1025E00068017901A9E0F694E794D794C794AA9575
:1025F000D1F7B7E1000F111F221F331FBA95D1F792
:102600000C291D292E293F29040D151D261D371DB6
:10261000CD84DE84EF84F8888CEBC81A8DEDD80A5F
:1026200086EDE80A8BE0F80AC80CD91CEA1CFB1CF2
:102630004A015B0180949094A094B094802A912ADE
:10264000A22AB32A84249524A624B7248C0C9D1C8A
:10265000AE1CBF1C7501640186E0CC0CDD1CEE1CB9
:10266000FF1C8A95D1F79AE1B694A7949794879422
:102670009A95D1F78C289D28AE28BF28800E911EF0
:10268000A21EB31EC9A4DAA4EBA4FCA499E6C91A3D
:10269000D10895EDE90A9CEBF90AC40ED51EE61E99
:1026A000F71EB301A2014095509560957095482999
:1026B00059296A297B2940275127622773274C0D06
:1026C0005D1D6E1D7F1D6A017B01EAE0CC0CDD1CE7
:1026D000EE1CFF1CEA95D1F7F6E1769567955795C4
:1026E0004795FA95D1F74C295D296E297F29480D28
:1026F000591D6A1D7B1D2996CCACDDACEEACFFAC40
:102700002997A9E5CA1AACEDDA0AABE6EA0AA4E50C
:10271000FA0AC40CD51CE61CF71C280139014094A8
:10272000509460947094442A552A662A772A482443
:1027300059246A247B244C0C5D1C6E1C7F1C730185
:102740006201AFE0CC0CDD1CEE1CFF1CAA95D1F79A
:10275000B1E17694679457944794BA95D1F74C2891
:102760005D286E287F28440E551E661E771EC9A060
:10277000DAA0EBA0FCA0B7ECCB1ABFE5DB0ABCE605
:10278000EB0AB3E0FB0AC00ED11EE21EF31E950158
:102790008401009510952095309504291529262946
:1027A000372904271527262737270C0D1D1D2E1D19
:1027B0003F1D680179018BE0F694E794D794C794A4
:1027C0008A95D1F795E1000F111F221F331F9A95AB
:1027D000D1F70C291D292E293F29040D151D261D71
:1027E000371D2196CCACDDACEEACFFAC2197EDE310
:1027F000CE1AE6EADE0AE4EAEE0AEAE9FE0AC80CC4
:10280000D91CEA1CFB1C4A015B0180949094A094A3
:10281000B094802A912AA22AB32A84249524A6243B
:10282000B7248C0C9D1CAE1CBF1C75016401E6E036
:10283000CC0CDD1CEE1CFF1CEA95D1F7FAE1B69436
:10284000A79497948794FA95D1F78C289D28AE2861
:10285000BF28800E911EA21EB31EC98CDA8CEB8C91
:10286000FC8CFEE6CF1AF3E3DF0AF3EFEF0AF0E7A2
:10287000FF0AC40ED51EE61EF71EB301A201409545
:10288000509560957095482959296A297B294027D8
:102890005127622773274C0D5D1D6E1D7F1D6A0138
:1028A0007B01AAE0CC0CDD1CEE1CFF1CAA95D1F725
:1028B000B6E17695679557954795BA95D1F74C2926
:1028C0005D296E297F29480D591D6A1D7B1DCDA8E4
:1028D000DEA8EFA8F8AC83E8C81A8BE0D80A80E13C
:1028E000E80AF108C40CD51CE61CF71C28013901C4
:1028F0004094509460947094442A552A662A772A0A
:10290000482459246A247B244C0C5D1C6E1C7F1CBB
:10291000730162018FE0CC0CDD1CEE1CFF1C8A955C
:10292000D1F791E176946794579447949A95D1F7AB
:102930004C285D286E287F28440E551E661E771E83
:10294000C988DA88EB88FC889FE2C91A92EAD90A1A
:102950009BE7E90A9AE7F90AC00ED11EE21EF31EB0
:10296000950184010095109520953095042915292D
:102970002629372904271527262737270C0D1D1D43
:102980002E1D3F1D68017901EBE0F694E794D79482
:10299000C794EA95D1F7F5E1000F111F221F331FED
:1029A000FA95D1F70C291D292E293F29040D151D53
:1029B000261D371DCDA4DEA4EFA4F8A8A1EBCA1AEA
:1029C000A1E8DA0AA7E5EA0AA0E9FA0AC80CD91CC4
:1029D000EA1CFB1C4A015B0180949094A094B09483
:1029E000802A912AA22AB32A84249524A624B724D3
:1029F0008C0C9D1CAE1CBF1C75016401A6E0CC0CA8
:102A0000DD1CEE1CFF1CAA95D1F7BAE1B694A79481
:102A100097948794BA95D1F78C289D28AE28BF2823
:102A2000800E911EA21EB31E2D968CAD9DADAEAD37
:102A3000BFAD2D9780529941A34DB140840F951F92
:102A4000A61FB71FB301A2014095509560957095E0
:102A5000482959296A297B2940275127622773274A
:102A6000840F951FA61FB71F6C017D014AE0CC0C97
:102A7000DD1CEE1CFF1C4A95D1F7AC01BD01E6E15F
:102A80007695679557954795EA95D1F74C295D2935
:102A90006E297F29480D591D6A1D7B1D8DA19EA1A0
:102AA000AFA1B8A58C5E9C4BAE4FBC45840D951D67
:102AB000A61DB71D2801390140945094609470946C
:102AC000442A552A662A772A482459246A247B24D2
:102AD000840D951DA61DB71D6C017D01FFE0CC0C7A
:102AE000DD1CEE1CFF1CFA95D1F72C013D01A1E184
:102AF0007694679457944794AA95D1F74C285D280B
:102B00006E287F28440E551E661E771E25968CADB6
:102B10009DADAEADBFAD25978F559E4EA74FB14B26
:102B2000800F911FA21FB31F95018401009510957E
:102B3000209530950429152926293729042715279A
:102B400026273727800F911FA21FB31F6C017D011D
:102B50001BE0F694E794D794C7941A95D1F78C01AB
:102B60009D0185E1000F111F221F331F8A95D1F7A8
:102B70000C291D292E293F29040D151D261D371D41
:102B80008D8D9E8DAF8DB8A18E579148AC4AB840BF
:102B9000880D991DAA1DBB1D4A015B01809490946C
:102BA000A094B094802A912AA22AB32A842495243E
:102BB000A624B724880D991DAA1DBB1D6C017D019B
:102BC000E6E0CC0CDD1CEE1CFF1CEA95D1F74C01B5
:102BD0005D01FAE1B694A79497948794FA95D1F79A
:102BE0008C289D28AE28BF28800E911EA21EB31EE1
:102BF00089AD9AADABADBCAD8B5C9D40A54CB244EC
:102C0000840F951FA61FB71FB301A20140955095D1
:102C100060957095482959296A297B2940275127B1
:102C200062277327840F951FA61FB71F6C017D01B4
:102C30004AE0CC0CDD1CEE1CFF1C4A95D1F7AC0120
:102C4000BD01E6E17695679557954795EA95D1F7E9
:102C50004C295D296E297F29480D591D6A1D7B1D50
:102C60008D899E89AF89B88D85549D42A842B54D06
:102C7000840D951DA61DB71D28013901409450945F
:102C800060947094442A552A662A772A4824592445
:102C90006A247B24840D951DA61DB71D6C017D0142
:102CA000FFE0CC0CDD1CEE1CFF1CFA95D1F72C01CB
:102CB0003D01A1E17694679457944794AA95D1F782
:102CC0004C285D286E287F28440E551E661E771EF0
:102CD00089A99AA9ABA9BCA98F569C42A947B4411E
:102CE000800F911FA21FB31F9501840100951095BD
:102CF00020953095042915292629372904271527D9
:102D000026273727800F911FA21FB31F6C017D015B
:102D10001BE0F694E794D794C7941A95D1F78C01E9
:102D20009D0185E1000F111F221F331F8A95D1F7E6
:102D30000C291D292E293F29040D151D261D371D7F
:102D400061968CAD9DADAEADBFAD6197880D991DFF
:102D5000AA1DBB1D61968CAF9DAFAEAFBFAF619793
:102D600089819A81AB81BC81800F911FA21FB31F03
:102D700089839A83AB83BC830D811E812F81388523
:102D8000040D151D261D371D0D831E832F833887C7
:102D900089859A85AB85BC85840F951FA61FB71FB3
:102DA00089879A87AB87BC87E796AEADBFADE797BB
:102DB000A05CBF4FE796BFAFAEAFE797B0E42B1A6A
:102DC000310811F00C94600761960CAD1DAD2EAD6D
:102DD0003FAD6197E996AEADBFADE99718960D93FB
:102DE0001D932D933C931B9709811A812B813C8164
:102DF0001C960D931D932D933C931F970D811E815F
:102E00002F81388550960D931D932D933C935397A6
:102E100009851A852B853C8554960D931D932D931A
:102E20003C935797E7968EAD9FADE797C858DF4F15
:102E30000FB6F894DEBF0FBECDBFDF91CF911F91CB
:102E40000F91FF90EF90DF90CF90BF90AF909F9049
:102E50008F907F906F905F904F903F902F9008954C
:102E60000F931F93CF93DF93EC01062F142F60E095
:102E70008E850E94CC023C852D858091170A88237F
:102E800081F09FB7F8948091170A813081F58DB356
:102E90008093A8024DB38091AC02809584238DBBB2
:102EA0009FBF3CBD2DBD0EBD00000DB407FEFDCF84
:102EB0008EB51EBD00000DB407FEFDCF1EB580917E
:102EC000170A882351F09FB7F8942091170A809130
:102ED000A802213079F48DBB9FBF61E08E850E94EE
:102EE000CC02812FDF91CF911F910F910895909384
:102EF000A802D7CF8FBFF1CFAF92BF92CF92DF9210
:102F0000EF92FF920F931F93CF936093031F7093E1
:102F1000041F8093051F9093061F6B017C01FF0C1B
:102F2000CC08DC2C76019B01AC016C2D7C2D8C2D0A
:102F30009C2D03E10E943B2DA12CE8E4BE2EF8EE6F
:102F4000CF2EDD24D394E12CF12C00E010E00E9480
:102F5000DE2CC22FC22ED32E7A01A7016627772737
:102F600066E88FEE9EE10E94301777276F2D5E2D69
:102F70004D2D67E88FEE9EE10E9430174C2F68E8D8
:102F80008FEE9EE1CF911F910F91FF90EF90DF9018
:102F9000CF90BF90AF900C94301740E00C94301756
:102FA000CF92DF92EF92FF920F931F93CF93DF9315
:102FB0006AE18FEE9EE10E94CD17C82FD0E069E153
:102FC0008FEE9EE10E94CD17682F880F770B880B3C
:102FD000990B0E94C22A20E030E040E85EE30E94A4
:102FE000212B0E94582C6B018B016091031F709163
:102FF000041F8091051F9091061F0E94C22A24ED94
:1030000030E843E45EE40E94BB2ABE0187FD10C0A5
:103010006D59710917FF0FC06C0D7D1DCB01DF913C
:10302000CF911F910F91FF90EF90DF90CF90089577
:10303000645A7109EFCF072E000C880B990B0E9480
:10304000C22A20EB32E748E85FE30E94212B0E946E
:10305000582CE4CF43E861E88FEE9EE10E943017E0
:1030600062E18FEE9EE10E94CD1783FFF9CF48E029
:1030700062E98FEE9EE10E94301781E090E00895B2
:10308000CF92DF92EF92FF926EE18FEE9EE10E946F
:10309000CD1782958F70CC24C394D12C02C0CC0C58
:1030A000DD1C8A95E2F70D2C000CEE08FF086DE19F
:1030B0008FEE9EE10E94CD1790E044E095958795B4
:1030C0004A95E1F78A30910534F5FC01EE0FFF1FB8
:1030D000E80FF91FEC5DFD4F608171818281082E40
:1030E000000C990B28EE33E040E050E00E94F52BF5
:1030F000C701B6010E94F52B21313105410551056B
:1031000074F04CE066EA8FEE9EE1FF90EF90DF9066
:10311000CF900C94301760E070E0CB01E3CF44E037
:10312000F1CFCF93DF93EC01863091052CF08D30F9
:10313000910534F5069731F545EC61EB8FEE9EE194
:103140000E9430174CE067EB8FEE9EE10E94301733
:10315000C6E0D0E06EE18FEE9EE10E94CD178F7049
:1031600094E0CC0FDD1F9A95E1F74C2F482B6EE9C8
:103170008FEE9EE10E943017DF91CF910C944018A2
:10318000CCE0D0E043EC61EB8FEE9EE10E94301783
:103190004AE067EB8FEE9EE10E943017DBCFCF93C2
:1031A000DF93EC01099714F0C8E0D0E06DE18FEEF9
:1031B0009EE10E94CD17C530D10514F4C5E0D0E0E2
:1031C0002497CC0FDD1F482F417F4C2B6DE98FEEEC
:1031D0009EE1DF91CF910C94301710920A1F10924C
:1031E000091F6DE18FEE9EE10E94CD17482F4E7FA3
:1031F0006DE98FEE9EE10C94301781E090E09093A2
:103200000A1F8093091F6DE18FEE9EE10E94CD178A
:10321000482F41606DE98FEE9EE10C943017CF93FB
:10322000DF93EC0141E861E88FEE9EE10E943017E8
:10323000CD2B99F00E94FD1840E06DE88FEE9EE1E5
:103240000E94301740E062EA8FEE9EE10E94301744
:1032500081E090E0DF91CF9108950E94ED18ECCFCE
:103260000F931F93CF93DF9366E08FEE9EE10E9452
:10327000CD17D82F67E08FEE9EE10E94CD17C82FA3
:1032800068E08FEE9EE10E94CD174C2F50E070E079
:1032900060E0762F652F542F44276D2B8A019B0108
:1032A000082BC901B80120E038E448EE51E00E9443
:1032B000B12C03E10E94562D2093200A3093210A5D
:1032C0004093220A5093230ADF91CF911F910F91CF
:1032D0000895CF92DF92EF92FF92CF93DF936091A8
:1032E0001C0A70911D0A80911E0A90911F0A0E946B
:1032F000C22A6B017C0120E030EC43EF55E40E94D0
:10330000BB2AD0E0C0E018160CF065C020E030E821
:1033100042E256E4C701B6010E94BB2AC1E0D0E0F8
:1033200018160CF058C020E030EC43E756E4C70113
:10333000B6010E94BB2AC2E0D0E018160CF04BC0C8
:1033400020E030E842EA56E4C701B6010E94BB2AF9
:10335000C3E0D0E018160CF03EC020E034E244EFA9
:1033600056E4C701B6010E94BB2AC4E0D0E018169B
:1033700094F520E034EE42E257E4C701B6010E9422
:10338000BB2AC5E0D0E0181634F520E034E244E76B
:1033900057E4C701B6010E94BB2AC6E0D0E0181668
:1033A000D4F420E034E244EF57E4C701B6010E94B0
:1033B000BB2AC7E0D0E0181674F420E034E244E7FA
:1033C00058E4C701B6010E94BB2AC9E0D0E0181634
:1033D00014F0C8E0D0E06DE18FEE9EE10E94CD17C1
:1033E0008F7044E0CC0FDD1F4A95E1F74C2F482B3E
:1033F0006DE98FEE9EE10E9430170E944018809187
:10340000501E882319F16DE18FEE9EE10E94CD17C9
:1034100090E034E0959587953A95E1F78A309105EB
:10342000E4F4FC01EE0FFF1FE80FF91FEC5DFD4F08
:1034300080819181A2810A2E000CBB0B80931C0A13
:1034400090931D0AA0931E0AB0931F0ADF91CF919B
:10345000FF90EF90DF90CF90089580E090E0DC0146
:10346000EDCF68E18FEE9EE10E94CD179FB7F894F3
:103470004091130850911408609115087091160836
:103480009FBF4093170850931808609319087093D2
:103490001A0880FF2AC081E08093B1028093B002B5
:1034A0008093AF028091AD029091AE022091B10263
:1034B000211108C02091B002211104C02091AF0257
:1034C000222301F18F309105B8F401969093AE025A
:1034D0008093AD0281E080934D1E80914C1E882325
:1034E000F1F061E08CE00C94CC021092B1021092E9
:1034F000B0021092AF02D6CF81E080934D1E809330
:103500004C1EEBCF009741F001979093AE02809351
:10351000AD0210924D1EE1CF10924C1EFACF0C94CA
:103520000B06CF93DF9362E18FEE9EE10E94CD17F1
:10353000C82F482F62E98FEE9EE10E943017C5FD2B
:103540002DC01092081F1092071F8091091F9091A3
:103550000A1F62E2892B09F463E18FEE9EE10E946B
:10356000CD17C82FD0E060E18FEE9EE10E94CD170D
:10357000482F6DE88FEE9EE10E943017E0910B1FFF
:10358000F0910C1F309711F0CE01199540E06DE8D5
:103590008FEE9EE1DF91CF910C943017DF91CF91A8
:1035A000089508950F931F93CF93DF93EC01E88163
:1035B000F9810084F185E02D1995892BB1F06DE03A
:1035C000CE010E94CD17082F60E0CE010E94CD17DA
:1035D000182F402F6DE8CE010E943017812F90E008
:1035E000DF91CF911F910F9108958FEF9FEFF8CF4B
:1035F000CF93DF93EC01E881F9810084F185E02D20
:103600001995892B69F0888D998D0196998F888FEE
:1036100060E0CE010E94CD1790E0DF91CF91089538
:103620008FEF9FEFFACFCF93DF93EC012097E1F07C
:1036300021978091AA029091AB02843F9140A0F41F
:103640008FEE9EE10E94F81A2091AA023091AB02FF
:10365000A9014F5F5F4F5093AB024093AA02225ED5
:103660003C4FF9018083E2CFDF91CF9108950F9312
:103670001F93CF93DF93EC018091190A811178C0D9
:103680008FEE9EE10E94F81A21974091000280FF80
:1036900055C09C0154E0359527955A95E1F72F7058
:1036A00033274F3FD1F41092AB021092AA0220931D
:1036B00000020E94D017909302028093010269E1F8
:1036C0008FEE9EE10E94CD178093A902CE01DF917B
:1036D000CF911F910F910C94131B2413E4CF0E94E0
:1036E000D0172091010230910202820F931F97FDA3
:1036F000019695958795909302028093010200911F
:10370000A90210E069E18FEE9EE10E94CD17800FC3
:10371000912F911D959587958093A902CE010E94C6
:10372000131B8FEF809300020E94D2050E94C205F6
:10373000DF91CF911F910F910C94E4044F3F39F02A
:103740001092AB021092AA028FEF809300020E94A7
:10375000D017909302028093010269E18FEE9EE1FF
:103760000E94CD178093A902CE010E94131BDCCFCB
:103770001092AB021092AA02EACFCF93DF93EC0132
:1037800063E10E94CD1790E0288D398D821B930B49
:10379000DF91CF910895AF92BF92CF92DF92FF92C7
:1037A0000F931F93CF93DF936C015B01EA0162E2F9
:1037B0000E94CD17F82E90E09C012C0F3D1F2F3F4B
:1037C000310529F020F0CFEFD0E0C81BD90B8501DF
:1037D000AC0EBD1E0A151B0541F0F80141918F0189
:1037E00060E8C6010E943017F5CF4C2F4F0D62EAFA
:1037F000C6010E943017CE01DF91CF911F910F912A
:10380000FF90DF90CF90BF90AF900895CF93DF935C
:103810001F92CDB7DEB76983DC01ED91FC91028088
:10382000F381E02D41E050E0BE016F5F7F4F1995BD
:103830000F90DF91CF91089590E080E008950C946F
:10384000DF2BCF938091150A811103C00E94ED18E0
:103850000CC0C091160ACC23C9F30E94FD184C2F4E
:1038600062EA8FEE9EE10E94301745E861E88FEE34
:103870009EE1CF910C9430178091501E882341F126
:103880008091B802843A89F440911602509117024F
:103890004F30510514F04EE050E057FD40E04067D6
:1038A00069E88FEE9EE10C943017893A89F44091D3
:1038B0001602509117024231510514F041E150E0D7
:1038C0004230510514F442E050E042504068E8CFE5
:1038D0000895CF92DF92EF92FF92CF93DF930E94F1
:1038E000B804D091501ED1117DC080911302811176
:1038F00084C1C0914B1ECC2309F47FC1C090200A23
:10390000D090210AE090220AF090230A61E0809191
:10391000FD1E0E94580361E08091FD1E0E94CC02B2
:103920008091FF1E9091001F8F3F9807C9F061E0C2
:103930000E94580360E08091FF1E0E94CC026AE062
:1039400070E080E090E00E94850461E08091FF1EBD
:103950000E94CC026AE070E080E090E00E94850462
:10396000DFB7F8948091180A811127C0EDE1F2E0E9
:103970008491E3E6F2E09491E82FF0E0EE0FFF1F70
:10398000EC54FE4FA591B491EC91E92321F461E050
:1039900085E30E94CC0261E085E30E9458038CB568
:1039A00080618CBD8CB580648CBD61E084E30E9435
:1039B000580361E083E30E9458038091180A8F5FE7
:1039C0008093180ADFBF62E48FEE9EE10E94CD175C
:1039D000823181F081E00E94500590E080E00E94F9
:1039E0004D06D0E08D2FDF91CF91FF90EF90DF90CB
:1039F000CF90089540E861E88FEE9EE10E94301775
:103A0000C701B6010E947C1740E06EE88FEE9EE190
:103A10000E94301740E06FE88FEE9EE10E94301761
:103A20006CE08FEE9EE10E94CD17482F43606CE85A
:103A30008FEE9EE10E94301744E066EA8FEE9EE131
:103A40000E94301740E869E88FEE9EE10E9430172F
:103A500041E861E88FEE9EE10E94301781E080939B
:103A6000501E0E943C1C0E94691980911A0A909174
:103A70001B0A0E94911880911402909115020E94D5
:103A8000CF180E9430196EE18FEE9EE10E94CD1793
:103A9000482F44606EE98FEE9EE10E94301787E365
:103AA0009BE190930C1F80930B1F60E08091011F9E
:103AB0000E94580340E060EC8FEE9EE10E943017B8
:103AC0002091011F3091021F80E02230310551F01A
:103AD00081E02330310531F0C9014297049788F421
:103AE00087E1821B2FB7F8948230E9F160F48823D4
:103AF00009F43FC0813071F082E08093170A80E0C2
:103B00000AC08FEFEFCF843091F178F18530A1F7C3
:103B100088E001C080E29091AC02892B8093AC02D6
:103B20008091170A811103C081E08093170A2FBF8B
:103B30002091011F3091021F22303105E1F481E90B
:103B40009AE1909304028093030280916A0083605B
:103B500080936A00EC9A0E94211C83E090E00E940E
:103B60000F06DC2F3FCF81E0D6CF82E0D4CF84E0B8
:103B7000D2CF80E1D0CF2330310569F481E99AE1D9
:103B8000909306028093050280916A008C60809376
:103B90006A00ED9AE0CFC90142970497E0F687E109
:103BA000821BE82FF0E0EE0FFF1FED5FFD4F21E9D4
:103BB0003AE131832083843091F08530B9F083304D
:103BC00039F080916900836080936900E89AC3CFDF
:103BD000809169008C6080936900E99ABCCF8091E4
:103BE0006900806380936900EA9AB5CF809169008B
:103BF000806C80936900EB9AAECF83E090E00E94E6
:103C0000EE05F0CE1F920F920FB60F9211240BB655
:103C10000F922F933F934F935F936F937F938F9365
:103C20009F93AF93BF93EF93FF9381E59EE10E9433
:103C30000702FF91EF91BF91AF919F918F917F917B
:103C40006F915F914F913F912F910F900BBE0F900D
:103C50000FBE0F901F9018951F920F920FB60F92E4
:103C600011240BB60F922F938F939F93EF93FF9393
:103C7000E091611EF091621E8081E091671EF091DB
:103C8000681E82FD1DC0908180916A1E8F5F8F73B8
:103C900020916B1E821741F0E0916A1EF0E0EF5A0E
:103CA000F14E958F80936A1EFF91EF919F918F91B6
:103CB0002F910F900BBE0F900FBE0F901F90189575
:103CC0008081F2CF1F920F920FB60F9211242F9383
:103CD0003F938F939F93AF93BF93809113089091DD
:103CE0001408A0911508B09116083091B30223E092
:103CF000230F2D3758F50196A11DB11D2093B30256
:103D00008093130890931408A0931508B093160895
:103D10008091B4029091B502A091B602B091B70221
:103D20000196A11DB11D8093B4029093B502A0939A
:103D3000B602B093B702BF91AF919F918F913F911F
:103D40002F910F900FBE0F901F90189526E8230F0C
:103D50000296A11DB11DD2CF1F920F920FB60F92E6
:103D600011240BB60F922F933F934F935F936F9352
:103D70007F938F939F93AF93BF93EF93FF93E091C4
:103D80001102F09112021995FF91EF91BF91AF913D
:103D90009F918F917F916F915F914F913F912F9163
:103DA0000F900BBE0F900FBE0F901F9018951F9293
:103DB0000F920FB60F9211240BB60F922F933F93D1
:103DC0004F935F936F937F938F939F93AF93BF9323
:103DD000EF93FF93E0910F02F09110021995FF917C
:103DE000EF91BF91AF919F918F917F916F915F9173
:103DF0004F913F912F910F900BBE0F900FBE0F90E0
:103E00001F9018951F920F920FB60F9211240BB6A8
:103E10000F922F933F934F935F936F937F938F9363
:103E20009F93AF93BF93EF93FF93E0910502F091BF
:103E300006021995FF91EF91BF91AF919F918F91DC
:103E40007F916F915F914F913F912F910F900BBE9A
:103E50000F900FBE0F901F9018951F920F920FB6E4
:103E60000F9211240BB60F922F933F934F935F93B2
:103E70006F937F938F939F93AF93BF93EF93FF9332
:103E8000E0910302F09104021995FF91EF91BF9127
:103E9000AF919F918F917F916F915F914F913F91E2
:103EA0002F910F900BBE0F900FBE0F901F90189583
:103EB0001F920F920FB60F9211240BB60F922F93F1
:103EC0003F934F935F936F937F938F939F93AF93A2
:103ED000BF93EF93FF93E0910D02F0910E021995BD
:103EE000FF91EF91BF91AF919F918F917F916F91D2
:103EF0005F914F913F912F910F900BBE0F900FBE8E
:103F00000F901F9018951F920F920FB60F921124C9
:103F10000BB60F922F933F934F935F936F937F93C3
:103F20008F939F93AF93BF93EF93FF93E0910B0217
:103F3000F0910C021995FF91EF91BF91AF919F9174
:103F40008F917F916F915F914F913F912F910F9042
:103F50000BBE0F900FBE0F901F9018951F920F92DF
:103F60000FB60F9211240BB60F922F933F934F93DE
:103F70005F936F937F938F939F93AF93BF93EF93D1
:103F8000FF93E0910902F0910A021995FF91EF91D8
:103F9000BF91AF919F918F917F916F915F914F9161
:103FA0003F912F910F900BBE0F900FBE0F901F905F
:103FB00018951F920F920FB60F9211240BB60F9205
:103FC0002F933F934F935F936F937F938F939F9321
:103FD000AF93BF93EF93FF93E0910702F091080234
:103FE0001995FF91EF91BF91AF919F918F917F9123
:103FF0006F915F914F913F912F910F900BBE0F905A
:104000000FBE0F901F9018951F920F920FB60F9230
:1040100011240BB60F922F933F934F935F936F939F
:104020007F938F939F93AF93BF93CF93EF93FF9320
:104030008091B202811127C081E08093B202C4E175
:1040400081E59EE10E94F101892BD9F08FB7F894A8
:104050004091471E5091481E2091431E3091441EAE
:104060004217530721F54091491E50914A1E209155
:10407000451E3091461E42175307C9F48FBFC150E9
:10408000F9F61092B202FF91EF91CF91BF91AF91EB
:104090009F918F917F916F915F914F913F912F9160
:1040A0000F900BBE0F900FBE0F901F901895409170
:1040B000491E50914A1E2091471E3091481E2150A2
:1040C000310942175307D1F28FBF81E59EE10E946B
:1040D000CF012FB7F894E091491EF0914A1E8083DA
:1040E0004091491E50914A1E8091451E9091461E56
:1040F0004817590751F48091431E9091441E9093A4
:104100004A1E8093491E2FBFBACF8091491E9091BD
:104110004A1E0196F4CF80EC90E00E94760286E081
:1041200090E00E9476028091501E90E00E947602FC
:1041300080EC90E00C94760288E198E00FB6F89459
:10414000A895809360000FBE909360000E94EA05DE
:104150000E940B06FBCF1F93CF93DF93EC01162F2A
:104160000E94DF2B181739F0612FCE01DF91CF911C
:104170001F910C94E72BDF91CF911F910895E1E5FA
:10418000FEE11382128288EE93E0A0E0B0E0848327
:104190009583A683B78386E492E09183808385EC40
:1041A00090E09587848784EC90E09787868780EC01
:1041B00090E0918B808B81EC90E0938B828B82ECF2
:1041C00090E0958B848B86EC90E0978B868B118E9C
:1041D000128E138E148E81E08093EE1EEFEEFEE1C0
:1041E0001382128228E532E03183208390E59487A0
:1041F00085878AE090E09787868789E090E0918BB9
:10420000808B82E090E0938B828B148A158A168AC9
:10421000178A118E108E138E128E158E148E1482A4
:104220001582168217820895CF93DF93CDB7DEB73C
:10423000C859D1090FB6F894DEBF0FBECDBF789430
:1042400084B5826084BD84B5816084BD85B582609B
:1042500085BD85B5816085BD80916E00816080934C
:104260006E001092810080918100826080938100B5
:1042700080918100816080938100809180008160C5
:10428000809380008091B10084608093B100809120
:10429000B00081608093B000809191008260809333
:1042A00091008091910081608093910080919000B5
:1042B0008160809390008091A10082608093A10032
:1042C0008091A10081608093A1008091A000816015
:1042D0008093A000809121018260809321018091D0
:1042E0002101816080932101809120018160809370
:1042F000200180917A00846080937A0080917A0016
:10430000826080937A0080917A00816080937A0045
:1043100080917A00806880937A001092C100809129
:104320007B00877F80937B0080E480937C0080917A
:104330007A00806480937A0080917A0086FDFCCFB9
:104340008091780060917900762F682F072E000CFD
:10435000880B990B611571058105910511F00E947B
:10436000B22AE2E1F5E081E093E0DF019C011D92D9
:1043700021503040E1F7F093441EE093431EF09348
:104380004A1EE093491EF093481EE093471E82E1C7
:1043900098E09093461E8093451EE091611EF09137
:1043A000621E82E08083E0915D1EF0915E1E1082AD
:1043B000E0915F1EF091601E80E180831092691E83
:1043C000E091651EF091661E86E08083E091631E99
:1043D000F091641E808180618083E091631EF09182
:1043E000641E808188608083E091631EF091641E6A
:1043F000808180688083E091631EF091641E8081DB
:104400008F7D80831092900089E18093910080E8F5
:104410009EE3909397008093960080E280937100D2
:1044200061E08CE00E94580361E08DE00E94580337
:10443000EEE1F3E084EF91E0DF019C011D92215059
:104440003040E1F7E4E2FAE084E0DF011D928A9572
:10445000E9F7E8E2FAE080E094E1DF019C011D92D7
:1044600021503040E1F7ECEEF2E082E3DF01282F4B
:104470001D922A95E9F7F0933A1EE093391EF093C6
:10448000401EE0933F1EF0933E1EE0933D1E2CE144
:1044900033E030933C1E20933B1EEAEBF2E0DF0159
:1044A0001D928A95E9F7F0932C1EE0932B1EF09352
:1044B000321EE093311EF093301EE0932F1E8AEEE1
:1044C00092E090932E1E80932D1E85E090E09093B5
:1044D000FE1E8093FD1E84E090E09093001F809369
:1044E000FF1E82E090E09093021F8093011F809155
:1044F000111F811101C083E0282F80FF6FC182E06E
:104500008093B9028091B9028150823008F07BC259
:1045100083ED9FE00E941F1C833709F074C188E37C
:104520009FE00E941F1C833009F069C189E39FE06E
:104530000E941F1C8093B802982F9F7B943A29F009
:10454000993A19F08F3F09F05EC18AE39FE00E941B
:104550001F1C81508E3F08F056C18BE090E00E94F6
:104560007A2D6C018C01E8E3EE2EEFE0FE2EC70100
:104570000E941F1CF80181938F01FFEFEF1AFF0AC1
:1045800023E4E2162FE0F20691F780E190E00E942A
:104590007A2D8C0181E093E2A5E4B7E689879A87BA
:1045A000AB87BC8789E89BEAADECBFEE8D879E8721
:1045B000AF87B88B8EEF9CEDAAEBB8E9898B9A8B0D
:1045C000AB8BBC8B86E794E5A2E3B0E18D8B9E8B31
:1045D000AF8BB88F1D821E821F821886FE01E75A9C
:1045E000FF4F80E4DF011D928A95E9F7CE018F5AD3
:1045F0009F4F28E0FC0111922A95E9F72BE0F60184
:10460000DE01599601900D922A95E1F720E82CA33E
:10461000FE01B5962CE2DF011D922A95E9F748E5E7
:1046200050E060E070E049835A836B837C8328E527
:10463000FC01208340E450E0BE01675E7F4F80555F
:1046400091090E94800639852A859B858C85D80131
:104650003C9311962C93119712969C931297139654
:104660008C9313973D852E859F85888914963C935E
:10467000149715962C93159716969C931697179644
:104680008C93179739892A899B898C8918963C9332
:10469000189719962C9319971A969C931A971B960C
:1046A0008C931B973D892E899F89888D1C963C93FE
:1046B0001C971D962C931D971E969C931E971F96D4
:1046C0008C934801BB24B394C7010E941F1CF401C2
:1046D00091914F018913B12CFFEFEF1AFF0A23E5E7
:1046E000E2162FE0F20681F7C8010E94162EC601DD
:1046F0000E94162EBB2009F488C081E080934B1ED7
:104700008FED9FE00E941F1C833709F07EC084ED6F
:104710009FE00E941F1C90E090931B0A80931A0A4E
:1047200085ED9FE00E941F1C90E0909315028093FE
:10473000140286ED9FE00E941F1C90E090931702E8
:10474000809316028BED9FE00E941F1C182F8CEDAA
:104750009FE00E941F1C90E0B0E0A0E07C01DD24FF
:10476000CC24F12A8DED9FE00E941F1C182F8EEDA6
:104770009FE00E941F1CC82AD12AC092200AD09212
:10478000210AE092220AF092230A87ED9FE00E941C
:104790001F1C182F88ED9FE00E941F1C90E0B0E0C6
:1047A000A0E07C01DD24CC24F12A89ED9FE00E9469
:1047B0001F1C182F8AED9FE00E941F1CC82AD12AB7
:1047C000C0921C0AD0921D0AE0921E0AF0921F0AA3
:1047D00082E1809318020E94691C17C083E022FDC9
:1047E0008FCE23FF02C081E08BCE42E250E066E62E
:1047F00072E081E59EE10E9493010E9436068F7E61
:10480000803E09F493CE10924B1E812C34E1932EFE
:10481000412C512C32015394AA24A39454E1B52E77
:104820008091501E882309F407C22FB7F894809115
:10483000130890911408A0911508B09116082FBF85
:1048400040911708509118086091190870911A0842
:10485000841B950BA60BB70B0397A105B10510F0B0
:104860000E94311A80914F1E882309F415C11091BE
:104870004E1E111102C00E94311A80914D1E8111ED
:10488000D7C180914C1E8111D3C1112331F062E355
:1048900070E080E090E00E9485040E94311A8091CF
:1048A0004D1E8111F9C010924E1E80910F0A811188
:1048B000EBC081E080930F0A4FB7F89420913D1E22
:1048C00030913E1E80913F1E9091401E4FBF281791
:1048D000390709F4D9C0E0913D1EF0913E1E809148
:1048E0003B1E90913C1EE817F90709F093C0809198
:1048F000391E90913A1E90933E1E80933D1E20815A
:104900003181E0912F1EF091301E80912D1E9091EB
:104910002E1EE817F90709F084C080912B1E909194
:104920002C1E9093301E80932F1E00811181C80190
:104930000197843F914008F0BFCFEBE1F8E02B51A5
:104940003840C9018E0F9F1FB4010E948E2CDC01DC
:10495000A85DB54F8C918193CF018B519840801702
:10496000910778F38091501E882309F485C08091C7
:10497000190A81115DC00E94EA050E94632AA30101
:1049800092010E94F52B607F362E0F3F110510F02B
:10499000689430F890E080E00E940F19632D8FEE4C
:1049A0009EE10E94061C9BE1C92E98E0D92EEE24C0
:1049B000E394F12CD6016D916D018FEE9EE10E9482
:1049C000061CBFEFEB1AFB0AEFEFEE16F10471F4D1
:1049D0000E942A1890E080E00E940F19632D8FEE4C
:1049E0009EE10E94061CEE24E394F12CC6018B513B
:1049F000984080179107F0F20E942A180E94E6055D
:104A00000E94211C59CF10924B1E4EE150E069E8E4
:104A100072E0EFCEE0913D1EF0913E1ECF01029676
:104A20006ACFE0912F1EF091301ECF01029679CF10
:104A30000E94EA050F3F110519F010F00FEF10E08A
:104A40008091150A811116C090E080E00E940F1934
:104A5000BBE1EB2EB8E0FB2ED7016D917D018FEE0F
:104A60009EE10E94061CC7018B5198408017910758
:104A700098F3C2CFC801EACF82E00E94500585E0DA
:104A800090E00E944D0618CF10924F1E1092381ED3
:104A90001092371E10920F0A4FB7F8942091471EBC
:104AA0003091481E8091491E90914A1E4FBF281791
:104AB000390709F4ADC481E08093421EFF24F394CA
:104AC000AEEFEA2E4FB7F8942091471E3091481E62
:104AD0008091491E90914A1E4FBF2817390709F44B
:104AE00095C4E091471EF091481E8091451E90911B
:104AF000461EE817F90709F0FFC08091431E909108
:104B0000441E9093481E8093471E10818091411E41
:104B1000882309F480C4103C09F00FC18091190268
:104B200081117CC41092411E80913D1E90913E1EC9
:104B30004091391E50913A1E8417950761F42091D7
:104B40003F1E3091401E80913B1E90913C1E2817C5
:104B5000390709F4B7CF20913F1E3091401E809154
:104B60003D1E90913E1E02972817390709F4AACFDF
:104B70008091371E9091381E8115944108F0A2CF84
:104B80002091351E3091361E8091331E9091341E37
:104B9000019710F48FEF93E12817390709F4B9C092
:104BA0002817390708F0AFC0821B930B01960097B6
:104BB00009F488CF60914F1E6F5F60934F1EE091A4
:104BC0003F1EF091401E3183208360913F1E709103
:104BD000401E20913B1E30913C1E6217730709F066
:104BE0009BC05093401E40933F1EE091311EF091B8
:104BF000321E918380832091311E3091321E80912C
:104C00002D1E90912E1E2817390709F090C0809113
:104C10002B1E90912C1E9093321E8093311E8091FA
:104C2000331E9091341E9093361E8093351E4ACFCA
:104C300081E080934E1E30CF8091110A9091120A2C
:104C4000A091130AB091140A0196A11DB11D2091E3
:104C50004B1E222369F1893FEAE29E07A105B105B7
:104C600048F48093110A9093120AA093130AB09308
:104C7000140A12CF1092110A1092120A1092130AFB
:104C80001092140A6091EE1E81E0623018F06832D2
:104C900018F08FEF8093100A8091100A680F6093CC
:104CA000EE1E70E08CE00E9489030E94E605F4CEBF
:104CB000893FFAE29F07A105B10598F21092110A07
:104CC0001092120A1092130A1092140A6091EE1EAA
:104CD00081E0623018F0683218F08FEF8093100A8C
:104CE0008091100A680F6093EE1E70E08DE00E94C4
:104CF00089030E940B06D0CEE091471EF091481E1A
:104D0000CF010196FECEB501621B730B860F971F74
:104D10004ECF81E090E04ECF20913F1E3091401E5B
:104D20002E5F3F4F3093401E20933F1E5ECF8091F9
:104D3000311E9091321E02966ECF2091291E309125
:104D40002A1E243F81E0380708F0BCCE909119025A
:104D50002115310529F49E3F19F410931902B2CEA2
:104D6000911144C01B3D19F4F092281EABCE8091E6
:104D7000281E882349F01C3D21F01D3D19F41BED30
:104D800001C010EC1092281E80914F1E883108F04F
:104D900099CE8091371E9091381E8115944108F06C
:104DA00091CE8091371E9091381E01969093381EB7
:104DB0008093371E8091331E9091341E9C012F5F8B
:104DC0003F4F3093341E2093331E885D954FFC0176
:104DD00010838091331E9091341E8115944109F007
:104DE00071CE1092341E1092331E6CCE913009F0A9
:104DF0004AC01B3DD9F49093281E8091291E9091A2
:104E00002A1E049709F05ECE6091240A7091250A4B
:104E10008091260A9091270A0E94AA2C611571059B
:104E200081059105D9F40E9478054CCE8091281E09
:104E3000882349F01C3D21F01D3D19F41BED01C0F4
:104E400010EC1092281EC901019690932A1E80939F
:104E5000291E2C5D354FD9011C93CFCF6093200ABA
:104E60007093210A8093220A9093230A20911802BA
:104E70002131C9F62091501E2223A9F20E947C17ED
:104E80000E943019D0CF923009F048C01B3DD9F4B0
:104E9000F092281E8091291E90912A1E049709F0F5
:104EA00011CE6091240A7091250A8091260A909172
:104EB000270A0E94AA2C6115710581059105D9F474
:104EC0000E949D05FFCD8091281E882349F01C3D3E
:104ED00021F01D3D19F41BED01C010EC1092281EAD
:104EE000C901019690932A1E8093291E2C5D354F8F
:104EF000F9011083CFCF60931C0A70931D0A809331
:104F00001E0A90931F0A809118028131C9F6809180
:104F1000501E8823A9F20E946919D2CF9330A9F4B8
:104F20001F3F19F40E941A05CDCD123108F011E18E
:104F3000812F90E0909317028093160280911802BF
:104F4000813181F70E943C1CEDCF9430F9F41F3F72
:104F500019F40E943E05B6CD86E090E0163038F098
:104F6000812F90E08D30910514F08CE090E09093CB
:104F70001B0A80931A0A20911802213151F72091BF
:104F8000501E222331F30E949118E3CF9530F9F49B
:104F90001F3F19F40E942C0595CD85E090E0153057
:104FA00038F0812F90E08930910514F088E090E08E
:104FB000909315028093140220911802213151F729
:104FC0002091501E222331F30E94CF18E3CF993055
:104FD000B9F41093160A112381F0F092150A80ECAF
:104FE00090E00E94760289E090E00E947602612FB4
:104FF00081E59EE10E94290244C01092150AEFCF7C
:10500000963049F51F3F19F40E948B205BCD11119A
:105010001CC040E861E88FEE9EE10E9430179FB708
:10502000F8948091180A882319F081508093180A07
:105030008091180A811105C08CB58F7B8CBD1092B0
:10504000170A9FBF1092501EDFCF113009F03ACDE2
:105050000E94691CD9CF9132C9F480EC90E00E9483
:10506000760281E290E00E94760280E00E94640570
:1050700080E00E94640580E00E94640580E00E9458
:10508000640580EC90E00E9476021CCD923239F4E7
:1050900080EC90E00E94760282E290E0E4CF9332CE
:1050A00019F40E94D2050ECD973081F40E94B80405
:1050B00080EC90E00E94760287E090E00E94760209
:1050C0008091130290E00E947602DBCF903329F4A6
:1050D000812F90E00E940F06F5CC903491F48091DE
:1050E000501E10E0882331F06CE28FEE9EE10E94AA
:1050F000CD17182F80EC90E00E94760280E490E0BB
:1051000074CF983071F4133709F0DCCC80EC90E068
:105110000E94760288E090E00E94760286E490E0A9
:10512000D2CF9E30C1F4113089F41093190A80EC6B
:1051300090E00E9476028EE090E00E9476028091DC
:10514000190A882331F181E090E0BDCF1111EFCF32
:105150001092190AECCF9F30F9F480914F1E8831DC
:1051600080F48091371E9091381E8115944148F447
:1051700080EC90E00E9476028FE090E00E94760240
:10518000E2CF80EC90E00E9476028FE090E00E94F7
:10519000760290E080E097CF9935A9F4183F09F0A6
:1051A00091CC82E390E00E944D0608E31FE06FEF90
:1051B000C8010E94AB200F5F1F4F011520E11207AD
:1051C000B1F70E949C20953521F4183F09F07ACC64
:1051D000F8CF9135B1F480EC90E00E94760281E541
:1051E00090E00E94760208E31FE0C8010E941F1CA5
:1051F0000E9464050F5F1F4F011530E11307A9F7E7
:1052000040CF9235D9F51B3DE9F4F092281E8091EC
:10521000291E90912A1E029709F054CC0091250A6C
:105220001091240A83ED9FE00E941F1C833711F127
:10523000183C00F5812F90E0602F885C904F0E9411
:10524000AB2040CC8091281E882349F01C3D21F0E2
:105250001D3D19F41BED01C010EC1092281EC90170
:10526000019690932A1E8093291E2C5D354FD901FB
:105270001C93CDCF83E00E94500524CC903579F467
:1052800080EC90E00E94760280E590E00E94760239
:1052900081E090E00E94760287E190E014CF98349C
:1052A00059F480EC90E00E94760288E490E00E943D
:1052B000760280E990E007CF993459F480EC90E0D1
:1052C0000E94760289E490E00E94760282E990E0F2
:1052D000FACE933509F093C080914B1E882309F4D0
:1052E00089C08091501E882309F484C060911A0AF5
:1052F00084ED9FE00E94AB206091140285ED9FE059
:105300000E94AB206091160286ED9FE00E94AB20C8
:1053100060911C0A70911D0A80911E0A90911F0ACB
:10532000692F77278827992787ED9FE00E94AB2078
:1053300060911C0A70911D0A80911E0A90911F0AAB
:10534000BC018827992788ED9FE00E94AB206091DF
:105350001C0A70911D0A80911E0A90911F0A672FE6
:10536000782F892F992789ED9FE00E94AB206091CB
:105370001C0A8AED9FE00E94AB206091200A709188
:10538000210A8091220A9091230A692F7727882782
:1053900099278BED9FE00E94AB206091200A7091CD
:1053A000210A8091220A9091230ABC01882799271B
:1053B0008CED9FE00E94AB206091200A7091210A41
:1053C0008091220A9091230A672F782F892F99279D
:1053D0008DED9FE00E94AB206091200A8EED9FE052
:1053E0000E94AB2063E78FED9FE00E94AB208AE034
:1053F00090E070CE8AE090E00E94EE0563CB943599
:1054000009F060CB60E08FED9FE019CF1092421E53
:105410000E949B0205CA103C09F054CBF092411E39
:10542000E092190210922A1E1092291E4BCB8F92E5
:105430009F92AF92BF92CF92DF92EF92FF92CF9363
:10544000DF93EC01688179818A819B816115710507
:105450008105910521F464E279ED8BE597E02DE17A
:1054600033EF41E050E00E94F52B49015A019B01C6
:10547000AC01A7EAB1E40E94142C6B017C01ACEEF4
:10548000B4EFA50194010E94222CC60ED71EE81E7F
:10549000F91EF7FE06C081E0C81AD108E10880E8CD
:1054A000F80AC882D982EA82FB82C701B6019F77D7
:1054B000DF91CF91FF90EF90DF90CF90BF90AF90B2
:1054C0009F908F9008958F929F92AF92BF92CF92AC
:1054D000DF92EF92FF9260911A0270911B0280910D
:1054E0001C0290911D02611571058105910521F441
:1054F00064E279ED8BE597E02DE133EF41E050E098
:105500000E94F52B49015A019B01AC01A7EAB1E4C5
:105510000E94142C6B017C01ACEEB4EFA501940148
:105520000E94222CC60ED71EE81EF91EF7FE06C0EA
:1055300081E0C81AD108E10880E8F80AC0921A028E
:10554000D0921B02E0921C02F0921D02C701B6012C
:105550009F77FF90EF90DF90CF90BF90AF909F909C
:105560008F90089560931A0270931B0280931C021F
:1055700090931D0208950E94FD2A08F481E0089589
:10558000E89409C097FB3EF49095809570956195DD
:105590007F4F8F4F9F4F9923A9F0F92F96E9BB2793
:1055A0009395F695879577956795B795F111F8CF0F
:1055B000FAF4BB0F11F460FF1BC06F5F7F4F8F4F7A
:1055C0009F4F16C0882311F096E911C0772321F070
:1055D0009EE8872F762F05C0662371F096E8862F08
:1055E00070E060E02AF09A95660F771F881FDAF75F
:1055F000880F9695879597F90895990F0008550F8C
:10560000AA0BE0E8FEEF16161706E807F907C0F048
:1056100012161306E407F50798F0621B730B840B50
:10562000950B39F40A2661F0232B242B252B21F42A
:1056300008950A2609F4A140A6958FEF811D811DCA
:1056400008950E94342B0C94A52B0E94972B38F0C0
:105650000E949E2B20F0952311F00C948E2B0C941D
:10566000942B11240C94D92B0E94B62B70F3959F88
:10567000C1F3950F50E0551F629FF001729FBB2749
:10568000F00DB11D639FAA27F00DB11DAA1F649FE5
:105690006627B00DA11D661F829F2227B00DA11D98
:1056A000621F739FB00DA11D621F839FA00D611D1E
:1056B000221F749F3327A00D611D231F849F600D3F
:1056C000211D822F762F6A2F11249F5750409AF068
:1056D000F1F088234AF0EE0FFF1FBB1F661F771FF4
:1056E000881F91505040A9F79E3F510580F00C94BF
:1056F0008E2B0C94D92B5F3FE4F3983ED4F3869520
:1057000077956795B795F795E7959F5FC1F7FE2B5E
:10571000880F911D9695879597F9089597F99F673A
:1057200080E870E060E008959FEF80EC0895002429
:105730000A941616170618060906089500240A94F6
:1057400012161306140605060895092E0394000C7C
:1057500011F4882352F0BB0F40F4BF2B11F460FF0B
:1057600004C06F5F7F4F8F4F9F4F089557FD905834
:10577000440F551F59F05F3F71F04795880F97FB15
:10578000991F61F09F3F79F08795089512161306CF
:105790001406551FF2CF4695F1DF08C016161706FE
:1057A0001806991FF1CF8695710561050894089533
:1057B000E894BB2766277727CB0197F90895F999D5
:1057C000FECF92BD81BDF89A992780B50895262F06
:1057D000F999FECF1FBA92BD81BD20BD0FB6F894D6
:1057E000FA9AF99A0FBE01960895052E97FB1EF4BA
:1057F00000940E940C2C57FD07D00E94272C07FC18
:1058000003D04EF40C940C2C509540953095219576
:105810003F4F4F4F5F4F08959095809570956195DC
:105820007F4F8F4F9F4F08950E94492CA59F900D49
:10583000B49F900DA49F800D911D11240895B7FF72
:105840000C94142C0E94142C821B930B0895A1E23B
:105850001A2EAA1BBB1BFD010DC0AA1FBB1FEE1FEA
:10586000FF1FA217B307E407F50720F0A21BB30B35
:10587000E40BF50B661F771F881F991F1A9469F7B1
:1058800060957095809590959B01AC01BD01CF010D
:105890000895A29FB001B39FC001A39F700D811D09
:1058A0001124911DB29F700D811D1124911D089529
:1058B0000E945F2C6894B1110C94D92B08950E941A
:1058C000BE2B88F09F5798F0B92F9927B751B0F0A9
:1058D000E1F0660F771F881F991F1AF0BA95C9F774
:1058E00014C0B13091F00E94D82BB1E008950C940F
:1058F000D82B672F782F8827B85F39F0B93FCCF3C2
:10590000869577956795B395D9F73EF490958095F0
:10591000709561957F4F8F4F9F4F0895AA1BBB1BBA
:1059200051E107C0AA1FBB1FA617B70710F0A61B9F
:10593000B70B881F991F5A95A9F780959095BC01C0
:10594000CD010895EE0FFF1F881F8BBF0790F691C2
:10595000E02D1994692796276927782787277827C4
:105960000895E894DF93CF93FC01DB010E94492C5A
:105970007F936F93E9019A01AC01BF93AF933F937B
:105980002F93DF010E94492C26F46C1B7D0B820BA8
:10599000930B9E01EB01FC010E94712DAF91BF9111
:1059A0002F913F910E94712DBE01CF01F9012F91DE
:1059B0003F91CF91DF910895689401C0E8948F9250
:1059C0009F92CF93DF930E94EA2CDF91CF919F901B
:1059D0008F90089588249924F401E401B0E49F9302
:1059E000AA279A158B049C04ED05FE05CF05D00768
:1059F000A10798F4AD2FDC2FCF2FFE2FE92D982C87
:105A0000892E982F872F762F652F542F432F322FD3
:105A10002227B85031F7BF9127C01B2EBF91BB275B
:105A2000220F331F441F551F661F771F881F991FA2
:105A3000881C991CEE1FFF1FCC1FDD1FAA1FBB1F58
:105A40008A149B04EC05FD05CE05DF05A007B10710
:105A500048F08A189B08EC09FD09CE09DF09A00B64
:105A6000B10B21601A94E1F62EF49401AF01BE014E
:105A7000CD01000C0895002E083090F0982F872F4C
:105A8000762F652F542F432F322F22270850F4CF23
:105A9000220F331F441F551F661F771F881F991F32
:105AA0000A95B2F7002D089597FD1094002E083046
:105AB00098F00850232F342F452F562F672F782F1B
:105AC000892F912DF4CF15949795879577956795A4
:105AD00057954795379527950A95AAF71124002DD4
:105AE00008950E94492C460F571FC81FD91F08F45C
:105AF000319608950F931F93CF93DF9382309105D2
:105B000010F482E090E0E0910F1FF091101F30E060
:105B100020E0B0E0A0E0309799F42115310509F4B8
:105B20004AC0281B390B24303105D8F58A819B8166
:105B30006115710589F1FB0193838283FE0111C018
:105B4000408151810281138148175907E0F04817BD
:105B5000590799F4109761F012960C9312971396C7
:105B60001C933296CF01DF91CF911F910F91089531
:105B700000930F1F1093101FF4CF2115310551F022
:105B80004217530738F0A901DB019A01BD01DF017B
:105B9000F801C1CFEF01F9CF9093101F80930F1F31
:105BA000CDCFFE01E20FF31F819391932250310973
:105BB00039832883D7CF20910D1F30910E1F232BBF
:105BC00041F4209120023091210230930E1F209346
:105BD0000D1F20911E0230911F022115310541F445
:105BE0002DB73EB74091220250912302241B350B62
:105BF000E0910D1FF0910E1FE217F307A0F42E1B8A
:105C00003F0B2817390778F0AC014E5F5F4F241720
:105C1000350748F04E0F5F1F50930E1F40930D1F26
:105C2000819391939FCFF0E0E0E09CCFCF93DF93FF
:105C30000097E9F0FC01329713821282A0910F1FA6
:105C4000B091101FED0130E020E01097A1F4208109
:105C50003181820F931F20910D1F30910E1F281745
:105C6000390709F061C0F0930E1FE0930D1FDF911B
:105C7000CF910895EA01CE17DF07E8F54A815B81ED
:105C80009E0141155105B1F7E901FB83EA83499172
:105C90005991C40FD51FEC17FD0761F480819181E4
:105CA0000296840F951FE9019983888382819381ED
:105CB0009B838A83F0E0E0E012968D919C9113978C
:105CC0000097B9F52D913C911197CD010296820F65
:105CD000931F20910D1F30910E1F2817390739F699
:105CE000309751F51092101F10920F1FB0930E1F96
:105CF000A0930D1FBCCFD383C28340815181840FF9
:105D0000951FC817D90761F44E5F5F4F888199814D
:105D1000480F591F518340838A819B8193838283DB
:105D20002115310509F0B0CFF093101FE0930F1F3C
:105D30009ECFFD01DC01C0CF13821282D7CFF89431
:025D4000FFCF93
:105D4200FFDCFEB704B704B704B704B704B704B75F
:105D520004B704010500FF0011FE0100000000006D
:105D6200121F8000781E00A02800F03C0040510065
:105D7200127A00E4A20024F40048E80190D0032043
:105D8200A1070000000029029301C0017B02F1017A
:105D9200CF01E30100000000061CCB1B1C1CD11A22
:105DA200BD1BF81AD21A4572726F722C20696E648A
:105DB200657465726D696E61746520626F6F7420BF
:105DC200766563746F720D0A004572726F722C20D1
:105DD200696E636F727265637420626F6F7420768E
:085DE2006563746F720D0A0085
:00000001FF
